:030000000211E901
:03000B000200BE32
:03002B000203E0ED
:03005B0002052477
:0300730002051A69
:1000800002030406080C10182030406080020304AC
:1000900006080C101820304080FF0406080C1018C9
:1000A0002030406080A0C000000001010003020277
:1000B000010505020D0505050D0603050202C2AF87
:1000C000C0D0C0E0205A25302F02E47330601A05FA
:1000D00060C37405952540F2956040EE758A78E519
:1000E000257003758A000203D90203CC306306C26F
:1000F00093C295C29785258AC25AE525F4700221DC
:10010000BF0561306013206A19758B00D0E0D0D034
:10011000C293C295C297D2AF32C293C295C2970220
:1001200001AFD26EC26FE565601CC3E561149565D1
:100130004014C26ED26FC3E561956450030201AFF3
:100140007561000201AF206C14C293C295C297740E
:100150000AD5E0FDD292D294D2960201AFC293C2E8
:1001600095C297E53D20E22520E10D207502D2924F
:10017000307502D2960201AF20E005D2940201AFA1
:10018000207502D296307502D2920201AF20E1159D
:1001900020E00D207502D292307502D2960201AF96
:1001A000D2940201AF207502D296307502D29275B8
:1001B0008B00D0E0D0D0C293C295C297D2AF32D0DC
:1001C000E0D0D0D2AF3261CCE525600A207502D2F2
:1001D00093307502D297C29561CCE5256002D29525
:1001E000207502C297307502C29361CCE525600A82
:1001F000207502D297307502D293207502C29330D7
:100200007502C29761CC207502C292307502C29607
:10021000E525600A207502D293307502D2972075C9
:1002200002C296307502C292C29561CC207502C29C
:1002300092307502C296207502C296307502C29243
:10024000740AD5E0FDE525600A207502D293307569
:1002500002D297C29561CC207502C292307502C25B
:1002600096E525600A207502D293307502D297C2B6
:1002700094C29561CC207502C292307502C296C2BA
:1002800094740AD5E0FDE525600A207502D293300A
:100290007502D297C29561CCC294E5256002D295D1
:1002A000207502C292307502C296207502C2973044
:1002B0007502C29361CCC294207502C2923075025D
:1002C000C296740AD5E0FDE5256002D2952075023C
:1002D000C297307502C29361CCC294E5256002D208
:1002E00095207502C296307502C292207502C2979F
:1002F000307502C29361CCC294207502C2963075EB
:1003000002C292740AD5E0FDE5256002D2952075FF
:1003100002C297307502C29361CC207502C296303A
:100320007502C292E525600A207502D297307502E7
:10033000D293C294207502C293307502C29761CCE9
:10034000207502C296307502C292C294740AD5E03A
:10035000FDE525600A207502D297307502D2932000
:100360007502C293307502C29761CC207502C296A5
:10037000307502C292E525600A207502D297307569
:1003800002D293207502C292307502C29620750285
:10039000C293307502C29761CC207502C296307547
:1003A00002C292207502C292307502C296740AD5BA
:1003B000E0FDE525600A207502D297307502D293E0
:1003C000207502C293307502C29761CCE525F4F521
:1003D0008A758B00756000D25AD0E0D0D0D2AF328F
:1003E000C2AFC0D0C0E0D2D3C2CEE528600A741F2D
:1003F000552E60491528813D78007900E5803076DA
:1004000001F430E30278FF53DACF20760343DA2099
:1004100030760343DA10C2D8C269E580307601F441
:1004200030E30279FFC3E89970CE3059037528187C
:10043000741F552E60037528188858D268E5296006
:100440000415298150741F552E600543DA01C2D866
:1004500020680281E2E558F8C268741F552E6036A4
:100460007982B70431C3E894F0400374F0F8E8C42B
:0F047000540F28F87984B703028196C313C3137E
:10047F008721200802C313200A06C3C898F8819663
:10048F0028F8500374FFF8C3E8955F5003E55FF851
:10049F00E52C5406703D882230630AC3E522955C33
:1004AF004003855C227882B60429C3E52295244057
:1004BF001278A096400DE52426F52450097524FFE7
:1004CF000204D5852224852425C3E524955C4003A9
:1004DF00855C2520CF09D0E0D0D0C2D3D2AF32C2B5
:1004EF00CF7801E5286008741F552E70021528C3B8
:1004FF00E55894014005755B00A111E55B046002AE
:10050F00055BD0E0D0D0C2D3D2AF32C2AF53917F10
:10051F00C258D2AF32C2AFC0D0C0E0C0F0D2D3A861
:10052F00FBA9FCC2D8306902A18753DACF2076032A
:10053F0043DA1030760343DA20D269E58030760152
:10054F00F420E302A15B88268927E12753DACF2025
:10055F00760343DA2030760343DA10C2D8C26974C7
:10056F001F552E7002E10D7800E580307601F430D2
:10057F00E302E10D8858E10D53DACF20760343DA19
:10058F002030760343DA10C269205902C14153DA91
:10059F00CF20760343DA1030760343DA20C2D8D265
:1005AF006988538954C3E89551F8E99552F9E4FBEA
:1005BF007AFAC3E894C8E994005008E4D2E4FB7ACD
:1005CF000AC114C3E89468E994015008E4D2E3FB2C
:1005DF007A0FC114C3E894D0E994025008E4D2E230
:1005EF00FB7A1EC114C3E894A0E994055008E4D225
:1005FF00E1FB7A3CC114C3E89498E994085006E4EF
:10060F00D2E0FB7A78C3E89555FCE99556FD30E7C3
:10061F0008ECF42401FCEDF4FD7557007008C3ECF1
:10062F009A500375570188558956A853A954885174
:10063F008952C3E89526F8E99527F9307402C1E08D
:10064F00307302C1E0307202C1D9E9C313F9E81364
:10065F00F8307102C1D9E9C313F9E813F830700209
:10066F00C1D9E9C313FDE813FC205918C3EC941C3E
:10067F00ED9402400302070DED7009C3EC94C850CE
:10068F000302072774002077037896E624FAFEE426
:10069F003400FFC3EC9EFCED9FFD500678007900FF
:1006AF00C1E0C3EC94FFED9400400678FF7900C1E0
:1006BF00E0EC856CF0A4C5F0A2F733F879004003A5
:1006CF000206FC78FF79000206FCE9C313F9E81370
:1006DF00F830740EE9600278FFC3E81338F8E43499
:1006EF0000F9C3E894FFE99400400278FF8858D2DC
:1006FF0068205902E10D741FF4552E4BF52E752805
:10070F0018741F552E700375280A305902E127748B
:10071F001F552E600353DAFE752906741F552E7070
:10072F000375290AD0F0D0E0D0D0C2D3D2AF32793E
:10073F0001E1567903E156790AE156791EE15679BE
:10074F0064E15679C8E1567817E4D5E0FDD8FAD9B7
:10075F00F6227A147B7802077D7A107B8C02077D54
:10076F007A0D7BB402077D7A0B7BC802077DAC251F
:10077F007525017902B275E4C294D5E0FDE52560D7
:10078F0002D295D5E0FDC295D5E0FDD294D5E0FD1E
:10079F00E525600A207502D293307502D297E56D78
:1007AF00D5E0FD207502C293307502C2977496D5BD
:1007BF00E0FDD9C1EAF8D5E0FDD8FBDBB1C2948CDE
:1007CF002522C37C007D0075F00005F0EA33FAEBBB
:1007DF0033FB50F6EB13FBEA13FAC3E9FFE8FEE82D
:1007EF009AF8E99BF95004EFF9EEF8B3EC33FCED0E
:1007FF0033FDD5F0DFEDF9ECF822E889F08A20D24D
:10080F00D4F8A9F07B0030F70B7BFFF42401F8E953
:10081F00F43400F9E88520F0A4ADF0F8E98520F074
:10082F00A4AFF0FEED2EF974003FFA7C04C3EA1377
:10083F00FAE913F9E813F8DCF48BF030F70AE8F46F
:10084F002401F8E9F43400F9E889F0C2D4F8A9F0EA
:10085F00227882B604030208ECC3E55894014018CD
:0F086F00E54870377805C37994B702027812C351
:10087E00E53B9400E53C984020E5486009855E5DC7
:10088E007562FF756301852224E4F53FF540F5415D
:10089E00F542F543F5480208EC754801C37994E733
:1008AE009402601BE523F43333F913F8E954010481
:1008BE00F9E854FEC39440F8E99400F90208E8E51B
:1008CE0023F433333333F913F8E954070404F9E806
:1008DE0054F8C39440F8E99400F9883F894022E522
:1008EE0048603BC3E53C13F9E53B13F8C3E53F987D
:1008FE00F8E54099F9500CC3E89480E994FF40164E
:10090E00020928C3E8947FE994005003020928786D
:10091E007F7900020928788079FF8844894522E58D
:10092E00486058E5442541F8E5453542F9854520AE
:10093E00E4300701F43543FA30E709C3EA94F04096
:10094E001502096AC3EA940F500302096A78FF7907
:10095E00FF7A0F02096A780079007AF0C3E52495D0
:10096E005C5006E52460092183E54520E70D2183CF
:10097E00E54530E706884189428A4322E5487003FF
:10098E000209ED789EE6FAC3E54433F8E54533F9FE
:10099E001109E930E70BC3E89480E994FF40132175
:1009AE00C4C3E8947FE99400500221C4787F790093
:1009BE0021C4788079FFE820E715C3E52398F84035
:1009CE0009C3E8940140030209EB78010209EBE840
:1009DE00F424012523F840030209EB78FF88462210
:1009EE00E5487003020A4F789FE6FAA842A9431120
:1009FE0009E930E70CC3E89401E994FF4016020AB6
:100A0E0026C3E894FFE994005003020A2678FF7982
:100A1E0000020A26780179FFE920E715C3E546981A
:100A2E00F84009C3E894014003020A4D7800020A17
:100A3E004DE8F424012546F84003020A4D78FF885C
:100A4E002422020AE77883E6F520120F6275E890F9
:100A5E00E5E820ECEDA8BDA9BE120FFA7568307559
:100A6E006900C3740013FD743013FC74302CFC74D5
:100A7E00003DFDECFAEDFBC3E89AE99B4014E568F6
:100A8E002430F568E5693400F569EA2CFAEB3DFB94
:100A9E0080E5AE68AF69C3E56913F9E56813F8C37D
:100AAE00E913F9E813F8E56828F566E56939F5679D
:100ABE007A03C3E913F9E813F8DAF7AA201A7009D2
:100ACE00756800756900020AE71AEA6008EE28FEEA
:100ADE00EF39FFDAF88E688F692275E890227883F5
:100AEE00E6FFE5E820ECF7A8BDA9BE056AC3E56AF6
:100AFE0094084052756A00E97007E56B601B020BA3
:100B0E001BC3E8956B6010E56B5006600C14020B6E
:100B1E00270460F9020B27E56BF56BC394A8F84028
:100B2E0021755CC0C3E89405F84017755C80C3E876
:100B3E009405F8400D755C40C3E89405F8400375C4
:100B4E005C0075BB0122C3E56AB4070375BB1E22A8
:100B5E0030610278323062027878E52C5406601FDC
:100B6E00E879A187F0A4C5F0A2F733F8C3E8955C45
:100B7E004002A85C882288248825306102885E2283
:100B8E00788FE6FFC3EF94055018C3EF94045020FE
:100B9E00C3EF94035028C3EF94025030C3EF940177
:100BAE0050387533A075340F75353C75360561F6C2
:100BBE007533C075341275354075360661F675336A
:100BCE00707534177535D075360761F675334C75FB
:100BDE00341D7535C475360961F6753328753423A1
:100BEE007535B875360B61F685334F853450753BC8
:100BFE0000753C0822A84FA950020C0EA849A94A1C
:100C0E00759100C3E498F594E499F595759104D225
:100C1E005875C820A8CCA9CD75C824AA39AB3A8876
:100C2E0039893AC3E89AF8E99BF9AA3BAB3CC3EB86
:100C3E0013FDEA13FCC3ED13FDEC13FCC3EA9CFA9F
:100C4E00EB9DFBEA28FAEB39FB8A3B8B3C400122F9
:100C5E00753BFF753CFF223058028165759100C3CC
:0F0C6E00E4954BF594E4954CF595759104D258A7
:100C7D00227892E6FF7E10305B027F053063047FA1
:100C8D00037E00A93CA83B7A04C3E913F9E813F8E5
:100C9D00DAF7C3E89EF8E99400F94009C3E8940235
:100CAD00E9940050047802E4F9E9FBE8FAC3E9138A
:100CBD00FDE813FCC3EF9403602EEF20E00DE82C4C
:100CCD00F8E93DF9ECFAEDFB020CE2E828F8E93918
:100CDD00F97A02E4FBC3EF9403400D8A4D8B4E88E5
:100CED0049894A8C4B8D4C22884D894E8A498B4AB5
:100CFD008C4B8D4C22305802A102759100C3E495A6
:100D0D003BF594E4953CF595759104D25822753ECA
:100D1D0000752000020D2A753E00752040D2AF05EA
:100D2D003E20580122759D00759C00E53CC313C300
:100D3D0013F8086036306A06C313C313F808C3E806
:100D4D00940A4002780A306D08C3E8940440027892
:100D5D0004C3E53C94084013759D02759C02C3E5E0
:100D6D003C94104006759D03759C03205803D2AF2B
:100D7D0022791E206D02790AD2AF0000C2AF205A2F
:100D8D000A793C206D027914306FE0306302797876
:100D9D00C3E58B9940D5E59E7005E59B020DAEE54B
:100DAD009AF45440B52002A12AD8C0D2AF22C25B1A
:100DBD00789CE6146007E53E147002D25B30630B3D
:100DCD000538205810753800020DE220580715819E
:100DDD00158102174D22759100C3E4954DF594E4EC
:100DED00954EF595759104D25822AE25305B4F780E
:100DFD00A3E6FFBF010BD25C752500C293C295C25D
:100E0D0097916A305C03752500305802C110BF02FE
:100E1D000BD25C752500C293C295C29778A2B6011C
:100E2D000D916A305C03752500305802C130BF0347
:100E3D000BD25C752500C293C295C297B1E3305CAD
:100E4D0003752500305802C14B305B04C25C8E2502
:100E5D0022C2AFC294206A03020E8090031A206C46
:100E6D0012306E0F207502C296307502C292740A4E
:100E7D00D5E0FD207502D292307502D296759F3362
:100E8D00759E00753D02D2AF22C2AF206A03020EDD
:100E9D00B89002D9306E17C294207502C296307583
:100EAD0002C292740AD5E0FD020EBB9001DA2075E4
:100EBD0002C297307502C293305A06E5256002D200
:100ECD0095207503759E23307503759E22753D0320
:100EDD00D2AF22C2AF207502C292307502C29620E7
:100EED006A03020F02900298206C0A306E07C294BA
:100EFD00740AD5E0FD207502D296307502D292208B
:100F0D007503759E22307503759E23753D04D2AF12
:100F1D0022C2AF206A03020F40900257306E172095
:100F2D007502C292307502C296C294740AD5E0FD64
:100F3D00020F439001C8C295305A0EE525600A2074
:100F4D007502D293307502D297759F33759E0075D9
:100F5D003D05D2AF22C2AF207502C296307502C2D6
:100F6D0092206A03020F8C900206206C12306E0FD5
:100F7D00207502C292307502C296740AD5E0FDD278
:100F8D0094207503759E23307503759E22753D065D
:100F9D00D2AF22C2AF206A03020FCA90036B306E2C
:100FAD001F207502C292307502C296207502C2963C
:100FBD00307502C292740AD5E0FD020FCD9001EC9E
:100FCD00207502C293307502C297305A0EE5256026
:100FDD000A207502D297307502D293207503759E43
:100FED0022307503759E23753D01D2AF229001C647
:100FFD00C293C295C297C292C294C29622C3E54FC4
:10100D009535E55095365001227890E6FFC3EF9463
:10101D00055018C3EF9404501BC3EF9403501EC327
:10102D00EF94025021C3EF94015024C3E54F943C3B
:10103D00F8021065C3E54F9428F8021065C3E54F1B
:10104D00941AF8021065C3E54F9412F8021065C3A7
:10105D00E54F940AF8021065E5509400F9884F8920
:0F106D00502230580302106F2278847603788562
:10107C00760478867607788F76037890760578955F
:10108C00760278927603789B760D7893760578873E
:10109C007603789C76017888760178897601788257
:1010AC007604788C7601788D7600788E76B4789686
:1010BC007625789776D078987678789976C8789AD5
:1010CC007604789D7600227893E6FF756409756541
:1010DC0001C3BF0209756405756501021118C3BF10
:1010EC000309756405756502021118C3BF040975FF
:1010FC006405756503021118C3BF0506756409758F
:10110C006507C3BF06067564007565007887E6FF42
:10111C00C26CC3BF0302D26CC26BC3BF0402D26BDE
:10112C00C26A7418552D6002D26AC26E6002D26E09
:10113C00D26F6002C26FC2757888E630E102D27558
:10114C00C2767889E630E102D276C3EF9402600869
:10115C00758E01D26D021169758E00C26D22788078
:10116C00E61490008093789EF67881E614900080C7
:10117C0093789FF6120FFA22789BE61490008D93C9
:10118C0078A0F6120FFA227886E61490009A9378DB
:10119C00A1F6120FFA22789CE6149000A79378A27D
:1011AC00F6789CE6149000AC9378A3F6120FFA2212
:1011BC00227896E6FA7897E6FB3077047A007BFF84
:1011CC00C3EB9AFCC3948250027C82756C00056C54
:1011DC00EC856CF0A4C3E5F0948040F222C2D353AA
:1011EC00D9BF7581C043FF8012073E75EF0243B231
:1011FC0003E5B324044002F5B37580FF75A40075B4
:10120C00F1FE75D4F775900275A5FC75F2FC75D5D9
:10121C000075A0FD75A60275F30275D60075B0FFBA
:10122C0075A70175F4FF75E241120FFAE4F8F6D8D0
:10123C00FD117612177D11D3316A3184319331A2AD
:10124C0031BC31BD7898866D120FFA75885075894E
:10125C000275C82475910475D840120752120761A3
:10126C0012074A12076812074A12076F12074A122E
:10127C001CCD12075212075212074E75A82275B8D0
:10128C000275E69075F610759B80759D03759A80B6
:10129C00759C0375D10E75BC5875BB0175BA1F755D
:1012AC00E88012073ED2AF120A5043DA01C2D8C20C
:1012BC0069120752753001D2597A05E55770027AD6
:1012CC0005120742E558C3940240EEE52E541F85E3
:1012DC005A59F55AB559E2DAE2C25953DACF2076A7
:1012EC000343DA2030760343DA10C2D8C2691207FE
:1012FC004E1207427802741F552E70027800C3E517
:10130C00589840EDC2AF120761120761120761D203
:10131C00AF120752754700120742788CE6C394014E
:10132C0050030213ECE530C3940150030213EC7428
:10133C001F552E6035C3E55894FF50030213ECC2C1
:10134C00AF120776D2AF12074EC3E558940150EF97
:10135C00C2AF120761120746120761D2AF12074ED5
:10136C00C3E55894FF40E9021D527F05D27731BD89
:10137C0012074EC2AFC27731BDC3E558947FD2AFCE
:10138C004068C2AF120776D2AFDFE1C3E5589405CF
:10139C007897F6120752121819121CD57F0AD277B9
:1013AC0031BD12074EC2AFC27731BDC3E558947F31
:1013BC00D2AF50E8C2AF120761120746120761D2D2
:1013CC00AFDFDBE55824057896F612075212181990
:1013DC00121D0412074EC3E55894FF40F6021D522D
:1013EC00C3E5589547400385584712074EC3E55847
:1013FC00940140026123C2AF1207761207761207DE
:10140C0076D2AF120752753000E4F531F532053162
:10141C00E531F470360532789AE678281460127843
:10142C005014600D78A014600878F01460037532C5
:10143C0000C3E53298401415327899866DC2AF120C
:10144C000776D2AF7898866D12074E120742E528C0
:10145C007008741F552E700241C3C3E558940640A2
:0F146C00AD12074EE52870030212C3120FFAE407
:10147B00F522F523F524F525755CFF7885865FF558
:10148B003FF540F541F542F543F56AF548F52BF587
:10149B002CF55B120B8E756A0875BB1E12073E127C
:1014AB000AE8E5E820ECFBA8BDA9BEE97001F888C5
:1014BB006B120AEC756A0875BB1E7895E630E00373
:1014CB0002150A7887E6FE760211D37887EEF6D2FC
:1014DB0061C2AF120B5E85225C85225DD2AFC26109
:1014EB00752500756200756301D260D26375380093
:1014FB00120F62120FA0120C0A120B8E0216337807
:10150B0087E6FE76037893E6FD760511D37887EEB2
:10151B00F67893EDF6D260D261D26E120F62120F93
:10152B00A0120B5E12073E120E5E12073E12073E12
:10153B00120E96120742120EE012074212074212C7
:10154B000F1E120746120F6212074212073EC261AC
:10155B00D262120AE8120AEC120B5E756A0875BBAE
:10156B001E120FA0120C03120C7E110A116F120E19
:10157B005E120C03120C7E110A116F120E96120CD6
:10158B0003120C7E110A116F120EE0120C03120CD7
:10159B007E110A116F120F1E120C03120C7E110A10
:1015AB00116F120F62120C03120C7E110AC3E54F5E
:1015BB009535E5509536400C116FC3E558940150A5
:1015CB009102174D116FC2627887E6FE760211D336
:1015DB007887EEF685225C855E5D855E25756200FB
:1015EB00756301D263753800C2AF207502C29230A9
:1015FB007502C296207502C296307502C292742D86
:10160B00D5E0FDD2AF120FA0120C0A120C65120C12
:10161B007E120D02756A0075BB0102163311D312CF
:10162B000FA0756A0075BB01120D24120DBB120DB4
:10163B00E3120860120DF7120E5E120C0A120C6503
:10164B00120C7E120D02120D1B120DBB120DE312AA
:10165B0008ED120DF7120E96120C0A120C65120CF5
:10166B007E120D02120D24120DBB120DE312092D69
:10167B00120DF7120EE0120C0A120C65120C7E12F0
:10168B000D02120D1B120DBB120DE312098A120D66
:10169B00F7120F1E120C0A120C65120C7E120D02A1
:1016AB00120D24120DBB120DE31209EE120DF712DF
:1016BB000F62120C0A120C65120C7E120D02120D27
:1016CB001B120AE8120DBB120DE3120AEC120DF7F6
:1016DB00120FA0120C0A120C65120C7E120D0230A6
:1016EB00632A755CFF755DFF756200756301C3E569
:1016FB00389464400AC263D264753714021717C357
:10170B00E5589401400302163302174D306419E576
:10171B0037147005C264021628F537C3E5589401D7
:10172B00400302163302174DC3E55B9482501374CA
:10173B001F552E7004E5286009C3E53C94F0500258
:10174B00C133120FFA7887E6FE760211D37887EE53
:10175B00F6E4F522F523F524F525F55FC2601207B3
:10176B003E120FFA741F552E7006E528700241C306
:10177B008115901A0D7820121C00E520B45A0CA389
:10178B00121C00E520B4A50302179E11761218193E
:10179B0002181878827604901A077884121C00A31A
:1017AB0008121C00A308121C00A308121C00A3089B
:1017BB00121C00A308121C00A308A308A308121CE8
:1017CB0000A308A308A308121C00A308121C00A363
:1017DB0008A308121C00A308121C00A308A30812DC
:1017EB001C00A308121C00A308121C00A308121C47
:1017FB0000A308121C00A308121C00A308121C0053
:10180B00A308121C00A308121C00901A2122C2AFBD
:10181B00121C3F121C19901A00740A121C05A37497
:10182B0004121C05A37410121C05901A077884125D
:10183B001C04A308121C04A308121C04A308121CEA
:10184B0004A308121C04A308121C04A308A308A3D6
:10185B0008121C04A308A308A308121C04A3081253
:0F186B001C04A308A308121C04A308121C04A346
:10187A0008A308121C04A308121C04A308121C04BF
:10188A00A308121C04A308121C04A308121C04A314
:10189A0008121C04A308121C04A308121C04121C1C
:0818AA0052121C30901A212299
:101A00000A0410FFFFFFFF0304070301015AA501A9
:101A1000FFFF0305FF0305FF0225D0FAFA040D01BD
:021A200000FFC5
:101A4000235467794B4631323041485623202020B9
:101A500023424C48454C4923463331302320202033
:101A60002020202020202020202020202020202076
:101C0000E493F622E6438F01538FFD75EF0275B71B
:101C1000A575B7F1F0538FFE22438F02438F0175F4
:101C2000EF0275B7A575B7F1901A0DF0538FFC222E
:101C3000901A0D745A9105901A0E74A59105227A86
:101C40003079D07820901A409100E520F709A3DA86
:101C5000F7227A3079D0901A40E7910509A3DAF992
:101C600022AB6EA86FBB01057984021CCABB0205BA
:101C70007985021CCABB03057995021CCABB040501
:101C80007986021CCABB0505798F021CCABB0605F2
:101C90007990021CCABB07057992021CCABB0805D1
:101CA000799B021CCABB09057993021CCABB0A05B1
:101CB0007987021CCABB0B05799C021CCABB0C05A8
:101CC0007988021CCA7989021CCAE8F7227C0512AD
:101CD0000752DCFB22C2AF12076112076812076FBE
:101CE00012077612074612076112076812076F1271
:101CF000077612074612076112076812076F12076C
:101D000076D2AF22C2AF12077612076F120768129F
:101D1000076112074612077612076F12076812074B
:101D20006112074612077612076F120768120761E1
:101D3000D2AF22AE6EAF6FC2AF120761120761124F
:101D40000761120746DEF2120776120746DFF8D265
:101D5000AF2291D591CD91CD756E01756F017570E2
:101D600000B1337C05AD58120752C3ED955870F59C
:101D7000C3E55894014009C3E55894FF4032A18E51
:101D8000916112181991D5C2AF75EF1291CDDCD5C2
:101D90000570C3E5709403500280C691CD056FE5D0
:101DA0006E149000B193F808C3E56F98500280AEAE
:101DB00091CD91CD056EC3E56E940E5002809C12BC
:0C1DC0001076121819C2AF75EF1291CD09
:00000001FF
